:100000000C946B050C94B3050C94B3050C94B305D8
:100010000C94B3050C94B3050C94B3050C94B30580
:100020000C94B3050C94B3050C94B3050C94540FC5
:100030000C94B3050C944F1D0C94B3050C94B305AC
:100040000C94B3050C94B3050C94B3050C94A81D43
:100050000C94B3050C94B3050C94B3050C940808E8
:100060000C94B3050C94B3050C94B3050C94B30530
:100070000C94B305BA0DE10DD90EE10DD90E2D0E7C
:10008000500ED90EA70EB60E77137713AF13AF131A
:100090002A145E14551655167514551606140614B2
:1000A0000F165516241642168800000000000000A6
:1000B0000400050006000700080009000A000B0004
:1000C0000C000D000E000F001000110012001300B4
:1000D0001400150016001700180019001A001B0064
:1000E0001C001D001E001F00200021002200230014
:1000F0002400250026002700280029002A002B00C4
:100100002C002D002E002F003000310000003300A5
:100110003400000036003700380082003A003B000F
:100120003C003D003E003F004000410042004300D3
:100130004400450046000000000049004A004E000F
:100140004C004D004B004F00500051005200000089
:100150005400550056005700580059005A005B00E3
:100160005C005D005E005F00600061006200630093
:100170000000650085006700680069006A000000F3
:10018000000000000000000000000000000000006F
:10019000890087008A008B00E000E100E200E300B4
:1001A0000000E500E600E700291E1F20212223248D
:1001B0002526272D2E742A2B141A0815171C180C07
:1001C00012132F3028041607090A0B0D0E0F3334B3
:1001D000311D1B0619051110363738752C764E4B1C
:1001E000494C52504F514A4D56545F6061555C5DC9
:1001F0005E57595A5B6762666377444568696A80EF
:10020000707172738080658048463A3B3C3D3E3F4A
:1002100040414243808080807939007A7880807BB9
:100220007F7E8080807D8080706339385F6C6564FC
:100230003A20253032580A007573625F6C65643A63
:1002400020253032580A0073656E642025303258FC
:100250003A20253032580A0073656E642039443ADA
:1002600020253032580A0025303258200073656E40
:10027000642037303A20253032580A0073656E64A6
:100280002039433A20253032580A000A4B657962FA
:100290006F6172642073746172742E0A000A555380
:1002A0004220636F6E666967757265642E0A000A84
:1002B0000A544D4B3A34386436393634342B2F4C8B
:1002C0005546410A0A003003500043003900380007
:1002D00020006B006500790062006F006100720011
:1002E0006400200063006F006E00760065007200FD
:1002F00074006500720000000E0374002E006D0093
:100300002E006B002E000000040309040902740093
:10031000040100A0320904000001030101000921C9
:10032000110100012240000705810308000A0904A9
:1003300001000103010200092111010001224D0009
:100340000705820308000A090402000103000000F7
:100350000921110100012236000705830308000A64
:100360000904030002030000000921110100012219
:100370002200070584032000010705040320000173
:100380001201100100000008EDFE019801010102B8
:1003900000010631FF0974A1010975150026FF004F
:1003A0009520750881020976150026FF00952075B5
:1003B000089102C005010980A101850216010026ED
:1003C00037001A81002AB700751095018100C00519
:1003D0000C0901A1018503160100269C021A0100E7
:1003E0002A9C02751095018100C005010902A10136
:1003F0000901A10005091901290515002501950527
:1004000075018102950175038101050109300931EA
:100410001581257F95027508810609381581257F8C
:10042000950175088106050C0A38021581257F950E
:100430000175088106C0C005010906A1010507195B
:10044000E029E715002501950875018102950175E0
:100450000881010508190129059505750191029585
:1004600001750391010507190029FF150026FF00FA
:10047000950675088100C0636F6E73756D65723A7D
:1004800020253034580A0073797374656D3A20253D
:100490003034580A000A002530325820006B657944
:1004A000626F6172643A20004C45443A2025303234
:1004B000580A0025583A2530386225730A000A2068
:1004C0002030313233343536370A00290A00257599
:1004D000002F002575005D2800256400200025649C
:1004E00000200025640020002564007C00253032B7
:1004F00058006D6F7573656B6579205B62746E7CF7
:10050000782079207620685D287265702F61636C91
:10051000293A205B006D6B5F776865656C5F746975
:100520006D655F746F5F6D6178203D2025640A0002
:100530006D6B5F776865656C5F6D61785F73706523
:100540006564203D2025640A006D6B5F74696D65EC
:100550005F746F5F6D6178203D2025640A006D6BCC
:100560005F6D61785F7370656564203D2025640A66
:10057000006D6B5F696E74657276616C203D20253D
:10058000640A006D6B5F64656C6179203D202564B1
:100590000A006D6B5F776865656C5F74696D655F98
:1005A000746F5F6D6178203D2025640A006D6B5F7C
:1005B000776865656C5F6D61785F737065656420F1
:1005C0003D2025640A006D6B5F74696D655F746F13
:1005D0005F6D6178203D2025640A006D6B5F6D6161
:1005E000785F7370656564203D2025640A006D6B3B
:1005F0005F696E74657276616C203D2025640A0027
:100600006D6B5F64656C6179203D2025640A000A8A
:1006100000257500363A20776865656C5F74696DF2
:10062000655F746F5F6D61783A20000A0025750080
:10063000353A20776865656C5F6D61785F737065CA
:1006400065643A20000A00257500343A2074696D0B
:10065000655F746F5F6D61783A20000A0025750050
:10066000333A206D61785F73706565643A20000AE3
:1006700000257500323A20696E74657276616C28C7
:100680006D73293A20000A00257500313A2064650F
:100690006C6179282A31306D73293A20000A092DBE
:1006A0002056616C756573202D0A004D3E004D2566
:1006B000643E20003F007365742064656661756C5C
:1006C000740A00433E200077686572652064656C9B
:1006D00074613A20637572736F723D25642C2077C4
:1006E0006865656C3D25640A53656520687474709F
:1006F0003A2F2F656E2E77696B6970656469612E7C
:100700006F72672F77696B692F4D6F7573655F6BBC
:100710006579730A000A092D204D6F7573656B6545
:1007200079202D0A4553432F713A09717569740A6E
:10073000313A0964656C6179282A31306D73290A70
:10074000323A09696E74657276616C286D73290A94
:10075000333A096D61785F73706565640A343A09EC
:1007600074696D655F746F5F6D61780A353A0977FA
:100770006865656C5F6D61785F73706565640A3686
:100780003A09776865656C5F74696D655F746F5F62
:100790006D61780A0A703A097072696E7420766128
:1007A0006C7565730A643A097365742064656661E3
:1007B000756C74730A75703A092B310A646F776E21
:1007C0003A092D310A706775703A092B31300A7079
:1007D00067646F776E3A092D31300A0A7370656568
:1007E00064203D2064656C7461202A206D61785F0F
:1007F0007370656564202A202872657065617420B5
:100800002F2074696D655F746F5F6D6178290A00D0
:100810003F004D3E2000433E20004C25640A000A64
:10082000092D20436F6E736F6C65202D0A4553436D
:100830002F713A09717569740A6D3A096D6F757394
:10084000656B65790A000A092D204D61676963208F
:100850002D0A643A0964656275670A783A09646525
:10086000627567206D61747269780A6B3A09646514
:10087000627567206B6579626F6172640A6D3A090F
:100880006465627567206D6F7573650A763A0976DF
:10089000657273696F6E0A733A0973746174757364
:1008A0000A633A09636F6E736F6C65206D6F6465E0
:1008B0000A302D343A096C61796572302D3428463E
:1008C00031302D4634290A506175733A09626F6FD1
:1008D000746C6F616465720A003F0074696D6572C3
:1008E0005F72656164333228293A202530346C58B0
:1008F0000A006B6579626F6172645F69646C653A66
:100900002025580A006B6579626F6172645F7072AE
:100910006F746F636F6C3A2025580A00686F7374A8
:100920005F6B6579626F6172645F6C6564732829BF
:100930003A2025580A000A092D20537461747573F2
:10094000202D0A004743433A20352E342E302041D3
:1009500056522D4C4942433A20322E302E302041FF
:1009600056525F415243483A2061767233350A004D
:100970004F5054494F4E533A204C554641204D4F0D
:100980005553454B45592045585452414B455920E4
:10099000434F4E534F4C4520434F4D4D414E442005
:1009A000343039360A004255494C443A20343864D0
:1009B00036393634342B202831333A31343A313019
:1009C000204465632020392032303230290A005615
:1009D00049443A2030784645454428742E6D2E6BA4
:1009E0002E29205049443A20307839383031285067
:1009F000433938206B6579626F61726420636F6E72
:100A000076657274657229205645523A20307830E6
:100A10003130310A00444553433A20636F6E7665A6
:100A20007274732050433938206B6579626F61723C
:100A3000642070726F746F636F6C20696E746F20C6
:100A40005553420A000A092D2056657273696F6E6C
:100A5000202D0A000A6D6F7573653A206F66660A6D
:100A6000000A6D6F7573653A206F6E0A000A6B6538
:100A700079626F6172643A206F66660A000A6B657C
:100A800079626F6172643A206F6E0A000A6D617458
:100A90007269783A206F66660A000A6D617472693D
:100AA000783A206F6E0A000A64656275673A206FB3
:100AB0006E0A000A64656275673A206F66660A000E
:100AC0000A0A626F6F746C6F616465722E2E2E203D
:100AD00000433E20000011241FBECFEFD4E0DEBF54
:100AE000CDBF04B603FE28C080915A0490915B04E8
:100AF000A0915C04B0915D048730904BA740B04B4F
:100B0000D9F410925A0410925B0410925C04109273
:100B10005D0414BE0FB6F894A895809160008861BA
:100B200080936000109260000FBE10920108109236
:100B30000008E0E0F8E3099511E0A0E0B1E0EEE79D
:100B4000FCE402C005900D92A833B107D9F724E068
:100B5000A8E3B1E001C01D92AA35B207E1F70E94F7
:100B6000D90A0C943D260C940000FF93EF93E0917A
:100B70003801F0913901309709F00995EF91FF9113
:100B80000895FC018591803011F0EFDFFBCF0895CF
:100B9000FF27E0E230E247FF0CC0419597FF09C014
:100BA000EDE26095709580959095611D711D811D98
:100BB000911D27FF02C0219530E350E2AA27660F5E
:100BC000771F881F991FAA1FA41710F0A41B6395F5
:100BD0005A95A9F7AA3008F0A95FA05DAF93F395E5
:100BE000611571058105910541F7ED3211F4EF931F
:100BF000F395F21718F43F93F395FBCF8F91B5DF80
:100C0000FA95E1F70895E991F9918591803021F005
:100C1000853219F0AADFF9CF089520E0E8945591C4
:100C20005532C1F3503311F4689455915A3348F456
:100C3000505390F3220F022E220F220F200D250F6A
:100C4000F4CF0EF4219589919991533619F35337C6
:100C500029F1533559F1BC0188279927E8945C366E
:100C600021F48991999168945591543639F446EF5D
:100C70007EF077FF0DC08FEF9FEF0AC055374AE037
:100C800039F0583540E121F0523642E009F008953C
:100C9000FF93EF937DDFEF91FF91B7CFFF93EF933A
:100CA000FC0181918030B9F360DFFBCFFF93EF93BC
:100CB00068DFF1CFDF93CF93CDB7DEB72596A3DF03
:100CC000CF91DF9108955C9AEFE9FFE03197F1F75A
:100CD00000C000000E9401088FE99FE00197F1F732
:100CE00000C000005C980895CF93CFEF0E94ED07FD
:100CF000C1508F3FFFEF9F0741F4EFE9FFE03197CD
:100D0000F1F700C00000C111F1CFCF910895EF922B
:100D1000FF920F931F93CF93DF93539A549A519A54
:100D20005B9A5C9A599A0E94D7075C9A5B9820E577
:100D30002A95F1F75B9A8FEF90E722E0815090407F
:100D40002040E1F700C000000CE712E08DE6E82E3D
:100D500082E0F82E8CE90E9463060E947406EC0182
:100D6000CF3F8FEFD80719F4EBE3F1E02DC080916E
:100D70003C0480FF0AC0DF93CF931F930F930E9420
:100D80005A060F900F900F900F90CA3FD10561F750
:100D900080E70E9463060E947406EC01CF3F8FEF4C
:100DA000D807C1F280913C0480FF0AC0DF93CF9343
:100DB000FF92EF920E945A060F900F900F900F90A3
:100DC000CA3FD10539F6D0CF119281E0EB34F80754
:100DD000D9F75C98DF91CF911F910F91FF90EF9021
:100DE0000895EF92FF920F931F93CF93DF930E948A
:100DF000ED07F82E082F192F0F3F8FEF180709F076
:100E00004EC080913A01882309F493C008E512E0AE
:100E100097E4E92E92E0F92E8DE90E9463060E9484
:100E20007406EC01CF3F8FEFD80721F410923A01FE
:100E300080E07FC080913C0480FF0AC0DF93CF93A5
:100E40001F930F930E945A060F900F900F900F90D0
:100E5000CA3FD10559F780913A010E9463060E946A
:100E60007406EC01CF3F8FEFD807B1F280913C04BC
:100E700080FF10C0DF93CF9380913A011F928F9330
:100E8000FF92EF920E945A060F900F900F900F90D2
:100E90000F900F90CA3FD10509F0BECFC7CF809108
:100EA0003C0480FF0CC09F93FF9287E692E09F93E3
:100EB0008F930E945A060F900F900F900F90E801A9
:100EC00083E0D695C7958A95E1F76F2D67708C2FD3
:100ED0008F7007FF14C00E948411882319F1CF700E
:100EE000DD27C55CDE4F0770112781E090E001C06F
:100EF000880F0A95EAF780959881892312C00E948D
:100F0000841181110FC0CF70DD27C55CDE4F0770E3
:100F1000112781E090E001C0880F0A95EAF79881D7
:100F2000892B88835C9A8AE68A95F1F700C05C98E1
:100F30008F2DDF91CF911F910F91FF90EF9008952A
:100F4000E82FF0E0E55CFE4F8081089580FD02C04F
:100F500090E701C091E790933A0181FF05C090911D
:100F60003A01946090933A0190913C0490FF0CC038
:100F70001F928F9388E392E09F938F930E945A066B
:100F80000F900F900F900F9080913C0480FF0EC047
:100F900080913A011F928F9388E292E09F938F9302
:100FA0000E945A060F900F900F900F90089583E3C0
:100FB0008093CC001092CD00E9ECF0E08081806954
:100FC0008083808188608083EAECF0E080818063A8
:100FD000808352985A9A7894089520914B01809179
:100FE0004C01821759F030E0F901E35BFE4F80813C
:100FF0002F5F3F4F20934B0190E008958FEF9FEFBD
:1010000008959091C80095FFFCCF8093CE0008957D
:101010001F920F920FB60F9211242F933F934F936D
:101020008F939F93EF93FF9380914C0190E09C01ED
:101030002F5F3F4F40914B01421741F03091CE005E
:10104000FC01E35BFE4F308320934C01FF91EF9155
:101050009F918F914F913F912F910F900FBE0F90C5
:101060001F901895809158030895CF93DF9300D077
:101070001F92CDB7DEB79C0180915104843019F5E1
:1010800093E099833B832A839093E9008FEF9091BB
:10109000E800815095FD06C095ED9A95F1F70000A6
:1010A0008111F5CF8091E80085FF0DC040E050E050
:1010B00063E070E0CE0101960E948B0C8091E80005
:1010C0008E778093E8000F900F900F90DF91CF9173
:1010D0000895CF93DF9300D01F92CDB7DEB7209154
:1010E0005104243031F522E02983805891099B83F3
:1010F0008A8383E08093E9008FEF9091E80081502C
:1011000095FD06C095ED9A95F1F700008111F5CF98
:101110008091E80085FF0DC040E050E063E070E0A2
:10112000CE0101960E948B0C8091E8008E7780930F
:10113000E8000F900F900F90DF91CF9108952091CC
:1011400051042430F1F422E02093E9002FEF309194
:10115000E800215035FD06C035ED3A95F1F7000065
:101160002111F5CF2091E80025FF0BC040E050E0B1
:1011700065E070E00E948B0C8091E8008E77809390
:10118000E8000895CF93DF9320915104243049F56E
:1011900021E02093E90021E8215059F03091E80046
:1011A00035FD07C0EFE3F1E03197F1F700C0000033
:1011B000F3CF2091E80025FF14C0EC0140E050E09F
:1011C00068E070E00E948B0C8091E8008E7780933D
:1011D000E80088E0FE01A0E5B3E001900D928A9559
:1011E000E1F7DF91CF910895CF93C0914F02C111E4
:1011F0000BC00E948D1D643C79408105910520F053
:1012000081E080934F02C1E08C2FCF910895FF922F
:101210000F931F93CF93DF93D82F0FB607FE83C092
:1012200080915104843081F08091030190E0019617
:101230002091050130E0822393232091040130E0C6
:101240008217930709F0C9C00E94F408811110C0E9
:101250008091030190E001962091050130E0822306
:1012600093232091040130E08217930709F0B5C061
:101270000E94811D8C01C091E900CF709091EC001B
:10128000892F817090FD80E8C82B84E08093E9006D
:1012900085E0F82E8091EB0085FD42C08091EB0047
:1012A00080FF3EC08091EE0087FF3AC0809104012C
:1012B00090910301981709F457C09091E80095FFA9
:1012C0008AC0E0910101F0910201E80FF11D208137
:1012D0008F5F909105018923809304012093F10091
:1012E0008091E80085FDE2CF8091E80080FFDECFAD
:1012F0008091E8008E778093E800F0920001D6CFCD
:101300008091030190E001962091050130E0822355
:1013100093232091040130E08217930709F448C019
:10132000CF70C093E90040910301842F90E00196B3
:101330002091050130E0822393232091040130E0C5
:101340008217930709F44CC0E0910101F09102016A
:10135000E40FF11DD083809103018F5F909105010F
:101360008923809303013CC08091E80085FF33C04E
:10137000D093F10081E09091F200992391F0909147
:10138000E80090FF0EC09091E80095FF03C0109216
:10139000F100F9CF9091E8009E779093E800F092E9
:1013A0000001882309F4ACCFCF70C093E90018C0C6
:1013B00080910001882309F4B3CF0E94811D9C0114
:1013C0008017910711F4890165CF90910001915028
:1013D00090930001F8CF80E0CECF40910301B4CFCD
:1013E00080E0DF91CF911F910F91FF900895809140
:1013F0005004811104C00E94F10E0C94440F089512
:10140000109250040895089542E061EC81E00E943A
:10141000040C42E061EC82E00E94040C42E061ECCA
:1014200083E00E94040C42E261EC84E00C94040C22
:1014300080915304833009F453C030F4813071F04B
:10144000823009F48CC008958A3009F478C08B305A
:1014500009F45EC0893009F09AC020C0809152041E
:10146000813A09F094C08091E800877F8093E8007A
:101470008091560490915704892B21F468E080E50F
:1014800093E003C060E080E090E070E00E94D80C40
:101490008091E8008B778093E80008958091520452
:1014A000813209F074C08091560490915704892BC1
:1014B00009F06DC08091E800877F8093E8008091FB
:1014C000E80082FD05C0809151048111F8CF5FC012
:1014D0008091F100809358038091E8008B7753C08E
:1014E00080915204813A09F052C080915604909143
:1014F0005704892B09F04BC08091E800877F8093C7
:10150000E8008091E80080FFFCCF8091100136C098
:10151000809152048132D9F58091560490915704FC
:10152000892BA9F58091E800877F8093E8000E94CD
:10153000390C80915404809310010C9427138091EE
:101540005204813221F58091E800877F8093E80082
:101550000E94390C8091550480935903089580911D
:101560005204813AA1F48091E800877F8093E800DB
:101570008091E80080FFFCCF809159038093F100B7
:101580008091E8008E778093E8000C94390C0895E0
:101590000E94121D80914F04882329F00E943B1D58
:1015A00081110C94EE0B089508950C94D40A0C94B8
:1015B000D40ACF9384B7877F84BF0FB6F894A895D9
:1015C00080916000886180936000109260000FBE7F
:1015D00090E080E80FB6F8948093610090936100EA
:1015E0000FBE87E099E00E94E51C86E091E00E9432
:1015F00019108FEA92E00E94C1050E94D70A0E944A
:10160000D8100E94F10E0E94440F78940E94DA10C4
:1016100080915104843029F00E94FE0F0E94D40A68
:10162000F7CF8DE992E00E94C1050E94D50A8BE8B0
:1016300092E00E94C105C4E080915104853019F404
:101640000E94C80AF9CF0E94DE102091E400309178
:10165000E50080914D0290914E022817390709F458
:1016600064C08091E4009091E50090934E028093D5
:101670004D020E94F408882309F457C08091510458
:10168000843009F052C08091E9008F702091EC0005
:10169000922F917020FD90E8892BC093E9009091E2
:1016A000EB0090FF3FC09091EE0097FF3BC0909100
:1016B000040120910301291709F12091E80025FF79
:1016C0001DC0E0910101F0910201E90FF11D30818F
:1016D0009F5F209105019223909304013093F100C4
:1016E0009091E80095FDE3CF9091E80090FFDFCF67
:1016F0009091E8009E779093E800D9CF9091F20006
:10170000992381F09091E80090FF0CC09091E8003F
:1017100095FF03C01092F100F9CF9091E8009E77F9
:101720009093E8008F708093E9000E94FE0F84CFB1
:10173000292F332723303105C9F060F421303105DA
:1017400081F02230310509F041C084E790E02CE0BF
:1017500033E040C021323105E1F02232310531F170
:1017600035C082E190E020E833E034C09927813031
:10177000910549F028F0029749F5E6ECF2E005C042
:10178000E8E0F3E002C0E8EFF2E0849190E09F012E
:1017900021C064307105D0F4660F771FFB01EB5D4B
:1017A000FE4F2081318189E090E014C064307105E2
:1017B00068F4FB01EE0FFF1FE35EFE4F20813181D5
:1017C000FB01E75EFE4F808190E004C080E090E086
:1017D00020E030E0FA0131832083089584E089BD60
:1017E00086E089BD09B400FEFDCF8091D8008F7DD1
:1017F0008093D8008091E00082608093E000809127
:10180000E00081FDFCCF0895982F953068F5909306
:10181000E900981739F07091EC002091ED0050919B
:10182000F00003C0242F762F50E021FD02C09F5FFF
:10183000ECCF3091EB003E7F3093EB003091ED0028
:101840003D7F3093ED003091EB0031603093EB0041
:101850007093EC002093ED005093F0002091EE0087
:1018600027FDE5CF80E008958F708093E90081E047
:1018700008958091520487FF11C08091E80082FD95
:1018800005C0809151048111F8CF11C08091E8000A
:101890008B770BC080915104882349F08091E80038
:1018A00080FFF8CF8091E8008E778093E80008955C
:1018B0002091E4003091E50095E64091EC00842F02
:1018C000817040FF23C08091E80080FD1DC08091A1
:1018D0005104882399F0853099F08091EB0085FDC3
:1018E00011C04091E4005091E5002417350729F319
:1018F000915011F09A01E1CF84E0089582E00895BB
:1019000083E0089581E0089580E008954091E80023
:1019100042FFDDCF0895CF92DF92EF92FF920F93B7
:101920001F93CF93DF93EC018B017A010E94580C37
:10193000811135C0E114F10439F0F7018081918102
:10194000081B190BC80FD91FC12CD12C011511056B
:1019500029F18091E80085FD18C08091E8008E771C
:101960008093E8000E94FE0FE114F10449F0F701B2
:1019700080819181C80ED91ED182C08285E00FC0BE
:101980000E94580C882311F30AC089918093F100BA
:1019900001501109FFEFCF1ADF0AD8CF80E0DF91A5
:1019A000CF911F910F91FF90EF90DF90CF9008950E
:1019B00020915804309159042617370748F06115D3
:1019C000710539F42091E8002E772093E80001C0DA
:1019D000B901FC0120E06115710561F180915104AC
:1019E0008823D9F18530D9F18091E80083FD39C091
:1019F0008091E80082FD2BC08091E80080FFEBCF52
:101A00008091F20090E06115710551F088309105E8
:101A100038F421912093F100615071090196F3CFC0
:101A200021E0089709F020E08091E8008E7780930C
:101A3000E800D1CF2111D2CF0AC080915104882370
:101A400061F0853061F08091E80083FD0AC08091EB
:101A5000E80082FFF2CF80E0089582E0089583E0FD
:101A6000089581E008952091580430915904261773
:101A7000370748F06115710539F42091E8002E7799
:101A80002093E80001C0B901FC0120E06115710557
:101A900079F180915104882309F43DC0853009F41F
:101AA0003CC08091E80083FD3AC08091E80082FD4F
:101AB0002CC08091E80080FFE9CF8091F20090E097
:101AC0006115710559F08830910540F424912093F7
:101AD000F1003196615071090196F2CF21E008972B
:101AE00009F020E08091E8008E778093E800CECF67
:101AF0002111CFCF0AC080915104882361F0853035
:101B000061F08091E80083FD0AC08091E80082FFC7
:101B1000F2CF80E0089582E0089583E0089581E0A7
:101B200008951F93CF93DF93CDB7DEB7AA970FB673
:101B3000F894DEBF0FBECDBFE2E5F4E08091F10086
:101B4000819324E0EA35F207C9F70E94180A8091D0
:101B5000E80083FF2EC18091520490915304492FD5
:101B600050E04A30510508F024C1FA01E65CFF4F0D
:101B70000C942326803821F0823809F01AC108C05D
:101B800080914E0490914F04992389F082600FC098
:101B9000809156048F70853008F00BC18093E90066
:101BA0008091EB0085FB882780F91092E9009091E5
:101BB000E800977F9093E8008093F1001092F10085
:101BC000D1C0282F2D7F09F0F4C0882319F082306E
:101BD00061F0EFC080915404813009F0EAC0933085
:101BE00009F080E080934F042EC08091540481114D
:101BF0002AC0809156048F702FEF280F243008F0F0
:101C0000D8C08093E9002091EB0020FF1CC09330E6
:101C100021F48091EB00806214C09091EB00906100
:101C20009093EB0021E030E0A90102C0440F551F62
:101C30008A95E2F74093EA001092EA008091EB0067
:101C400088608093EB001092E9008091E800877F24
:101C50008093E8000E94390CACC08111AAC0109199
:101C600054041F778091E3008078812B8093E300F8
:101C70008091E800877F8093E8000E94390C809172
:101C8000E80080FFFCCF8091E30080688093E30050
:101C9000111102C082E001C083E08093510489C029
:101CA0008058823008F085C080915404909155048A
:101CB0008C3D53E0950779F583E08A838AE2898336
:101CC0004FB7F894DE01139620E03EE051E2E32F97
:101CD000F0E050935700E49120FF03C0E295EF70CD
:101CE0003F5FEF708E2F90E0EA3010F0C79601C092
:101CF000C0968D939D932F5F243149F74FBF8091FC
:101D0000E800877F8093E8006AE270E0CE010196E8
:101D10000E94D80C16C06091560470915704AE0111
:101D20004F5F5F4F0E94980BBC01892B09F441C0A3
:101D30009091E800977F9093E80089819A810E94B2
:101D4000330D8091E8008B778093E80032C08038B3
:101D500081F58091E800877F8093E80080914D04B1
:101D60008093F1008091E8008E7772CF811121C0BD
:101D7000809154049091550499270297D4F480914E
:101D8000E800877F8093E8008091540480934D049D
:101D90000E94390C80914D04811106C08091E300AE
:101DA00087FD02C081E001C084E0809351040E945D
:101DB000040A8091E80083FF0AC08091E800877FD1
:101DC0008093E8008091EB0080628093EB00AA96FC
:101DD0000FB6F894DEBF0FBECDBFDF91CF911F913C
:101DE00008950E944E0F0E94510FE0EEF0E08081B6
:101DF00081608083E8EDF0E080818F77808319BC7B
:101E0000E3E6F0E0808181608083109250040895C1
:101E10000E944E0F0E94510F8091D8008F778093BF
:101E2000D8008091D80080688093D8008091D80035
:101E30008F7D8093D80084E089BD86E089BD09B498
:101E400000FEFDCF1092510410924D0410924F04E9
:101E500010924E0442E060E080E00E94040C809109
:101E6000E1008E7F8093E1008091E20081608093A9
:101E7000E2008091E20088608093E2008091E000BF
:101E80008E7F8093E0000895E3E6F0E080818E7F0E
:101E9000808381E0809350040C94080F1092E2003C
:101EA00008951092E10008951F920F920FB60F92BD
:101EB00011242F933F934F935F936F937F938F934F
:101EC0009F93AF93BF93EF93FF938091E10082FFC5
:101ED0000BC08091E20082FF07C08091E1008B7F00
:101EE0008093E1000E94FD0F8091E10080FF18C007
:101EF0008091E20080FF14C08091E2008E7F809389
:101F0000E2008091E20080618093E2008091D8003D
:101F100080628093D80019BC109251040E94000A7C
:101F20008091E10084FF30C08091E20084FF2CC0EA
:101F300084E089BD86E089BD09B400FEFDCF8091B3
:101F4000D8008F7D8093D8008091E1008F7E8093B0
:101F5000E1008091E2008F7E8093E2008091E200B8
:101F600081608093E20080914D04882311F084E029
:101F700007C08091E30087FD02C081E001C083E0DB
:101F8000809351040E94F7098091E10083FF24C0EF
:101F90008091E20083FF20C08091E100877F8093E1
:101FA000E10082E08093510410924D048091E100A1
:101FB0008E7F8093E1008091E2008E7F8093E2002B
:101FC0008091E20080618093E20042E060E080E086
:101FD0000E94040C0E94030AFF91EF91BF91AF9100
:101FE0009F918F917F916F915F914F913F912F9131
:101FF0000F900FBE0F901F9018950895CF9380916A
:1020000051048823A1F0C091E900CF709091EC00B9
:10201000892F817090FD80E8C82B1092E900809193
:10202000E80083FD0E94910DCF70C093E900CF912D
:10203000089590935F0380935E030895E0915E039B
:10204000F0915F03309721F00190F081E02D099429
:1020500080E00895EF92FF920F931F93CF93DF9349
:10206000E0915E03F0915F033097B1F18C01028043
:10207000F381E02D099580913C0482FF2DC080FF03
:1020800004C08DE994E00E94C105E80118E087E9E9
:10209000E82E84E0F82E80913C0480FF0BC08881FC
:1020A0001F928F93FF92EF920E945A060F900F900B
:1020B0000F900F90115021961111EDCF80913C049B
:1020C00080FF0AC085E994E0DF91CF911F910F91C5
:1020D000FF90EF900C94C105DF91CF911F910F916C
:1020E000FF90EF900895E0915E03F0915F033097C9
:1020F00021F00480F581E02D09940895CF93DF93BA
:1021000020915C0330915D032817390709F1909302
:102110005D0380935C03E0915E03F0915F03309771
:10212000B9F0EC010680F781E02D099580913C041F
:1021300082FF0EC080FF0CC0DF93CF9387E894E04E
:102140009F938F930E945A060F900F900F900F90BD
:10215000DF91CF910895CF93DF9320915A0330916F
:102160005B032817390709F190935B0380935A03A7
:10217000E0915E03F0915F033097B9F0EC010084C9
:10218000F185E02D099580913C0482FF0EC080FF0F
:102190000CC0DF93CF9387E794E09F938F930E94C7
:1021A0005A060F900F900F900F90DF91CF910895E6
:1021B0000C9483110E94781D0C948706BF92CF92D5
:1021C000DF92EF92FF920F931F93CF93DF9300D094
:1021D00000D01F92CDB7DEB70E94F10601E613E0F2
:1021E000F12C8F2D0E94A007B82EF801C080C826C0
:1021F00039F4F3940F5F1F4FF0E1FF12F2CF30C0BC
:1022000080913C0481FD0E949811D12CEE24E3942E
:102210008C2D8E21F9F0D982FA8291E08B2D8E21BE
:1022200009F490E09B830E94811D8160782F9D833B
:102230008C8349815A816B818D810E94CE114981A5
:102240005A816B817C818D810E94FD1CF801808107
:102250008E258083D394EE0CF8E0DF12D9CFC9CF5E
:102260008FEF89838A831B820E94811D8160782F72
:102270009D838C8349815A816B818D810E94CE110F
:102280000E94FC1C0E9430200E941E10909160034E
:10229000891741F10E941E108093600390913C04C5
:1022A00092FF0EC090FF0CC01F928F9388EA94E0BB
:1022B0009F938F930E945A060F900F900F900F904C
:1022C000809160030F900F900F900F900F90DF910F
:1022D000CF911F910F91FF90EF90DF90CF90BF9023
:1022E0000C940E1D0F900F900F900F900F90DF9198
:1022F000CF911F910F91FF90EF90DF90CF90BF9003
:1023000008950C94A6070895CF93C62F0E94A007A6
:1023100021E030E002C0220F331FCA95E2F790E0BF
:102320002823392381E0232B09F480E0CF910895FD
:10233000EF92FF920F931F93CF93DF938EEB94E076
:102340000E94C105C0E0D0E08DE2E82E81E0F82EC9
:1023500003EB14E08C2F0E94A0070E94EA1CFF925E
:10236000EF921F928F93DF93CF931F930F930E944F
:102370005A0621968DB79EB708960FB6F8949EBF61
:102380000FBE8DBFC031D10529F7DF91CF911F91CD
:102390000F91FF90EF90089508950895CF93DF93E4
:1023A000CDB7DEB72B970FB6F894DEBF0FBECDBF0B
:1023B000942F4F83252F588769877A878B874A8583
:1023C0005B85452B31F02F3F31F481E09F3F19F4BD
:1023D00003C081E001C080E080FD07C04F815885C7
:1023E00069857A858B850E94FD1CDE01119686E049
:1023F000FD0111928A95E9F785E0FE01379601907B
:102400000D928A95E1F749815A816B817C818D819A
:102410009E810E9453192B960FB6F894DEBF0FBE13
:10242000CDBFDF91CF910895CF93DF93882309F437
:102430008FC0C82F8EE78C0F833018F5C23829F073
:10244000C33831F0C4E0D7E405C0C2E0D9E302C02C
:10245000C1E0D3E50E941E108C2309F079C08D2FB6
:102460000E94471C0E94BF1C2FEF81EE94E0215078
:1024700080409040E1F700C000008D2F0E94641C56
:1024800010C08CEF8C0F813A20F080E58C0F8E32DB
:1024900060F48C2F0E945B2381115AC08C2F0E9404
:1024A000471CDF91CF910C94BF1C80E28C0F8830C9
:1024B00048F4C77081E001C0880FCA95EAF70E940E
:1024C000851CEFCF8BE58C0F833080F4C53A29F063
:1024D000C63A31F083E890E005C081E890E002C0A0
:1024E00082E890E0DF91CF910C947E1088E58C0F0C
:1024F000873170F5C83A89F0C93A91F0CA3A99F033
:10250000CB3AA1F0CC3AA9F0CD3AB1F0CE3AB9F03D
:10251000CF3AC1F080E090E017C082EE90E014C0A6
:1025200089EE90E011C08AEE90E00EC085EB90E05D
:102530000BC086EB90E008C083EB90E005C084EB15
:1025400090E002C087EB90E0DF91CF910C94AB104C
:10255000DF91CF910895CF93DF93882309F454C07E
:102560009EE7980F933008F5823829F0833831F0D0
:10257000C4E0D7E405C0C2E0D9E302C0C1E0D3E5BE
:102580000E941E108C2309F43FC08D2F0E94471C0F
:102590000E94BF1C2FEF81EE94E0215080409040BC
:1025A000E1F700C000008D2F08C09CEF980F913A12
:1025B00020F090E5980F9E3218F40E94641C0DC024
:1025C00090E2980F983068F4877091E001C0990FFD
:1025D0008A95EAF7892F0E948B1CDF91CF910C948A
:1025E000BF1C9BE5980F933030F480E090E0DF91C2
:1025F000CF910C947E10885A873130F480E090E0BF
:10260000DF91CF910C94AB10DF91CF910895882387
:1026100021F00E94851C0C94BF1C0895882321F092
:102620000E948B1C0C94BF1C08950E94A51C0E9444
:10263000741C0E94BF1C0E94D6200E94A31F80E031
:1026400090E00E947E1080E090E00C94AB100E941D
:10265000951C0C941513CF92DF92EF92FF920F937B
:102660001F93CF93DF9300D000D01F92CDB7DEB77A
:102670006C010E94101D811118C385E0F601DE0176
:10268000119601900D928A95E1F7F60140815181F2
:10269000238134812115310531F05F3F31F481E030
:1026A0004F3F19F403C081E001C080E080FDFDC20E
:1026B000F601F280E580E2948FE0E82249835A83B4
:1026C000FB82722F3D832C836F2D8D810E94BC1B5A
:1026D0008C010E94BB1B0E94AB1AE12FE295EF70A8
:1026E0008E2F90E0FC01EC5BFF4F0C942326812F92
:1026F000807F1F70882311F01295107FFF20B9F0A2
:10270000112329F0812F0E94981C0E94BF1C802F4A
:102710000F900F900F900F900F90DF91CF911F911E
:102720000F91FF90EF90DF90CF900C941412802FB8
:102730000E94AB12112309F4B8C2812F0E949E1C83
:102740000F900F900F900F900F90DF91CF911F91EE
:102750000F91FF90EF90DF90CF900C94BF1C812FD2
:10276000807F1F70803211F01295107F002319F0C6
:10277000013009F12BC0FF20A9F0EE2059F1F1E062
:10278000812FEF1228C00F900F900F900F900F9095
:10279000DF91CF911F910F91FF90EF90DF90CF903D
:1027A0000C94A81CEE2021F021E0E21609F47DC271
:1027B0000E94AB1C4DC0FF20E9F085E08E1508F4A7
:1027C00074C20E94821C812329F042C0FF20F1F1D3
:1027D000E11015C0812F0F900F900F900F900F9068
:1027E000DF91CF911F910F91FF90EF90DF90CF90ED
:1027F0000C94071394E09E1508F457C229C0F60103
:10280000858180FF13C08F708583E4CF003F09F47A
:1028100089C108F055C180E4800F803208F459C1A5
:10282000FF2009F4EAC1EE2009F49AC1802F0E942A
:102830001412093309F0DAC1FFEF21EE84E0F15000
:1028400020408040E1F700C000002FC2E110D7C156
:10285000812F59C1812F86958695837019F081301B
:10286000B9F023C2FF2019F0C801937002C080E0C4
:1028700090E00F900F900F900F900F90DF91CF91FD
:102880001F910F91FF90EF90DF90CF900C947E10EE
:10289000FF2019F0C801937002C080E090E00F9013
:1028A0000F900F900F900F90DF91CF911F910F918C
:1028B000FF90EF90DF90CF900C94AB10802FFF2013
:1028C00019F00E94B61E02C00E941E1F0F900F90AA
:1028D0000F900F900F90DF91CF911F910F91FF906C
:1028E000EF90DF90CF900C94A31F812F837009F09D
:1028F00070C0F110DAC1202F229526952770220F83
:10290000220F602F6F70862F90E0A0E0B0E06C0186
:102910007D01022E04C0CC0CDD1CEE1CFF1C0A94B1
:10292000D2F704FF12C08FE090E0A0E0B0E004C056
:10293000880F991FAA1FBB1F2A95D2F7BC01CD0192
:10294000609570958095909503C060E070E0CB0134
:102950001695169513701230B1F040F56C297D294B
:102960008E299F29113031F10F900F900F900F9009
:102970000F90DF91CF911F910F91FF90EF90DF901B
:10298000CF900C94D01A6C297D298E299F290F9005
:102990000F900F900F900F90DF91CF911F910F919B
:1029A000FF90EF90DF90CF900C94EA1A0E94D01A1B
:1029B000C701B6010F900F900F900F900F90DF910D
:1029C000CF911F910F91FF90EF90DF90CF900C94DB
:1029D000B61AFF2019F0812F817001C086958823D7
:1029E00009F463C1202F229526952770220F220F0C
:1029F000602F6F70862F90E0A0E0B0E06C017D0149
:102A0000022E04C0CC0CDD1CEE1CFF1C0A94D2F775
:102A100004FF12C08FE090E0A0E0B0E004C0880F97
:102A2000991FAA1FBB1F2A95D2F7BC01CD01609543
:102A300070958095909503C060E070E0CB0116958D
:102A4000169513701230B1F040F56C297D298E294E
:102A50009F29113031F10F900F900F900F900F9030
:102A6000DF91CF911F910F91FF90EF90DF90CF906A
:102A70000C94971B6C297D298E299F290F900F900C
:102A80000F900F900F90DF91CF911F910F91FF90BA
:102A9000EF90DF90CF900C94A91B0E94971BC70169
:102AA000B6010F900F900F900F900F90DF91CF9184
:102AB0001F910F91FF90EF90DF90CF900C94851BAA
:102AC000023F09F45EC008F449C0033F09F46CC03A
:102AD000A7CE902F9071E92E812F8F71FF2051F09A
:102AE0000E941E1B802FEE2019F08295807F73CEEE
:102AF0008F7071CE0E943F1B802FEE2019F08295BF
:102B0000807F01C08F700F900F900F900F900F90EB
:102B1000DF91CF911F910F91FF90EF90DF90CF90B9
:102B20000C940E13FF20A9F0E4E0EE1508F4BDC0EC
:102B3000812F8F710F900F900F900F900F90DF915A
:102B4000CF911F910F91FF90EF90DF90CF900C9459
:102B5000641BF5E0FE1508F4A8C0EACFFF2099F049
:102B6000812F8F710F900F900F900F900F90DF912A
:102B7000CF911F910F91FF90EF90DF90CF900C9429
:102B80001E1BFF2069F3812F8F710F900F900F9004
:102B90000F900F90DF91CF911F910F91FF90EF90C9
:102BA000DF90CF900C943F1BFF2089F0812F8F7115
:102BB0000F900F900F900F900F90DF91CF911F917A
:102BC0000F91FF90EF90DF90CF900C94091B0F9026
:102BD0000F900F900F900F90DF91CF911F910F9159
:102BE000FF90EF90DF90CF900C94041B033509F415
:102BF00023CE073409F059C01FCEEE2021F2802FDA
:102C00000F900F900F900F900F90DF91CF911F9129
:102C10000F91FF90EF90DF90CF900C94AB12412F6B
:102C20004F70602FC6010E942C1E0F900F900F90C6
:102C30000F900F90DF91CF911F910F91FF90EF9028
:102C4000DF90CF900C94061A01112FC0FF2069F17C
:102C50000E9427132FEF80E792E0215080409040A0
:102C6000E1F700C000000F900F900F900F900F90B1
:102C7000DF91CF911F910F91FF90EF90DF90CF9058
:102C80000C94CE1D412F4F70602FC6010F900F90F6
:102C90000F900F900F90DF91CF911F910F91FF90A8
:102CA000EF90DF90CF900C942F1E0F900F900F900D
:102CB0000F900F90DF91CF911F910F91FF90EF90A8
:102CC000DF90CF9008951F93CF93DF9300D000D073
:102CD0001F92CDB7DEB7942F4983252F5A836B837C
:102CE0007C838D834C815D81452B31F02F3F31F406
:102CF00081E09F3F19F403C081E001C080E0182FFC
:102D0000117080FD31C049815A816B817C818D8138
:102D10000E94BC1B292F22952F702C3030F42A30B2
:102D2000A0F42250223030F022C02C30C9F02F30D5
:102D3000B9F01DC0853A28F48430C0F4823028F4FC
:102D400015C090E2980F983088F0883E30F4803EAD
:102D500068F48450813A58F409C0803F41F406C0B9
:102D600093FB112710F903C010E001C011E0812F7F
:102D70000F900F900F900F900F90DF91CF911F91B8
:102D80000895CF93DF9300D000D01F92CDB7DEB768
:102D90000F900F900F900F900F90DF91CF910895AB
:102DA000CF93DF9300D000D000D0CDB7DEB726960A
:102DB0000FB6F894DEBF0FBECDBFDF91CF9108955F
:102DC000CF93DF93C091710380917203C817A1F074
:102DD000D0E0CE0166E070E00E94FE25FC01ED58D7
:102DE000FC4F4081518162817381848195810E9471
:102DF000D0162196C770E8CFDF91CF91089540910A
:102E0000A3035091A4036091A5037091A603809140
:102E1000A7039091A8030C94D0161F93CF93DF9330
:102E20008091A80382958F7009F05CC08091A50302
:102E3000882309F457C02091710310917203C09147
:102E4000A303D091A403A091A603B091A70381E0AE
:102E5000CF3F09F080E0482F211709F443C01097B5
:102E600021F0DF3F21F080E003C081E001C0842F2A
:102E700030E080FD33C0C90166E070E00E94FE25AD
:102E8000FC01ED58FC4F81818D1328C080818C138B
:102E900025C08281811122C0838194818A1B9B0B72
:102EA000883C9105D8F48091A8038F70806180934D
:102EB000A803C90166E070E00E94FE25FC01E85805
:102EC000FC4F90819F709061908383EA93E00E9411
:102ED0002B13DF91CF911F910C94E0162F5F3F4F82
:102EE0002770BACFDF91CF911F9108959F92AF9233
:102EF000BF92CF92DF92EF92FF920F931F93CF93E7
:102F0000DF93CDB7DEB761970FB6F894DEBF0FBE83
:102F1000CDBF8C0185E0F801DE011D9601900D9278
:102F20008A95E1F7F80140812181F280C380D48045
:102F30009091A3033091A4036091A6037091A7031D
:102F40006115710531F03F3F31F481E09F3F19F485
:102F500003C081E001C080E0F82FF1709F2E80FD5A
:102F600059C183EAA82E83E0B82EE090A503F601AC
:102F7000E61BF70BEE2009F4EDC08091A803582F53
:102F8000507FE83CF10508F0A7C0511156C023134B
:102F900013C0491311C0EF2CF1100EC08F70806167
:102FA0008093A8030E94FF16C5010E942B138091F5
:102FB000A803F801858364C1C114D10431F02F3F07
:102FC00031F481E04F3F19F403C081E001C080E09B
:102FD00080FD03C081E08F2502C080E090E0F82FE3
:102FE000F170EF2E80FF1FC0E091710330917203EA
:102FF000E31709F421C1F0E0CF0166E070E00E9420
:10300000FE25DC01AD58BC4F11968C911197281309
:1030100007C08C91481304C012968C91F81203C01B
:103020003196E770E5CFEF2CFF2009F429C180919C
:10303000A80381608093A80364C0231306C04913CA
:1030400004C0F11002C0F801A9C04D872E87FF8689
:103050007C2DD98AC88A522F6F2D89890E946316C8
:103060008823A1F1FF2091F12091A803822F82955E
:103070008F7090E0029774F08091A3039091A40365
:1030800098878F831986DB86CA862C87CE010796A0
:103090000E942B1386E0F801A3EAB3E001900D92A1
:1030A0008A95E1F70E940D170E94FF1612C02317A0
:1030B00051F14D872E87FF867C2DD98AC88A522FE1
:1030C0006F2D89890E94631681112CC0C8010E944E
:1030D0002B13EE24E394D4C05111E9CF7C2DD98A6F
:1030E000C88A522F6F2D89890E94C11683EA93E006
:1030F0000E942B1386E0F50111928A95E9F70E9450
:10310000FF16E12CBDC04913D4CFF110D2CFF80186
:103110008583C8010E942B1386E0F50111928A95E0
:10312000E9F7AEC0FF2091F22091A803822F82958B
:103130008F7090E002970CF4ADCF8091A303909133
:10314000A4039A8389831B82DD82CC822E83CE01E5
:1031500001969ECFE83CF10508F04CC0EF2CFF2013
:1031600009F4B4CF231330C049132EC02091A80313
:1031700020FD21C0822F82958F70482F50E041158D
:103180005105C9F0F80125834F30510541F08F5F9B
:10319000982F9295907F822F8F70892B8583C801FD
:1031A0000E942B1386E0F801A3EAB3E001900D9290
:1031B0008A95E1F72CC086E0F801A3EAB3E001901C
:1031C0000D928A95E1F75CC04D872E87FF867C2D96
:1031D000D98AC88A522F6F2D89890E94631681115E
:1031E00059CF8091A80381608093A803C8010E94F1
:1031F0002B1346C07C2DD98AC88A522F6F2D8989FE
:103200000E94C11686E0F50111928A95E9F70E94A5
:10321000FF1636C0FF2009F459CF4D872E87FF8651
:103220007C2DD98AC88A522F6F2D89890E946316F6
:10323000882309F44BCF2ECF7C2DD98AC88A522FF0
:103240006F2D89890E94BC1B292F22952F70223057
:1032500028F49F7039F0811105C00BC0243028F488
:103260009F7049F4805E883020F0C8010E942B13C3
:103270009E2CE92C05C0F8019581907F99F7F9CF34
:103280008E2D61960FB6F894DEBF0FBECDBFDF91D5
:10329000CF911F910F91FF90EF90DF90CF90BF9053
:1032A000AF909F900895CF93DF93CDB7DEB72C9763
:1032B0000FB6F894DEBF0FBECDBF4F835887698726
:1032C0007A878B879C87CE0107960E947617882382
:1032D000D1F09F8188852A853B85232B31F08F3F54
:1032E00031F481E09F3F19F403C081E001C080E028
:1032F00080FD6FC04F81588569857A858B859C8557
:103300000E94D01666C086E0FE013796DE01119657
:1033100001900D928A95E1F7FF81E8856A857B85AA
:103320006115710531F0EF3F31F481E0FF3F19F491
:1033300003C081E001C080E080FD4BC0809172033A
:1033400090E09C012F5F3F4F27703327409171031E
:1033500050E02417350709F443C0F983EA837D83DD
:103360006C8366E070E00E94FE25DC01AD58BC4F26
:1033700096E0FE01319601900D929A95E1F7209327
:1033800072030E94E01625C090E066E070E00E94A3
:10339000FE258D589C4F0E947617882371F18091ED
:1033A000710390E066E070E00E94FE25FC01ED589C
:1033B000FC4F4081518162817381848195810E949B
:1033C000D0168091710390E00196877099278093C1
:1033D000710380917103909172038913D5CF0DC051
:1033E0000E9427131092720310927103E3EAF3E034
:1033F00086E0DF011D928A95E9F72C960FB6F894C6
:10340000DEBF0FBECDBFDF91CF910895DF92EF9267
:10341000FF920F931F93CF93DF93FC01892B09F445
:1034200088C0E12CF12CDD24D394EF012196849106
:10343000853709F460C058F4843708F04EC08430F2
:1034400008F068C08130D1F0823071F172C08837E5
:1034500009F45BC050F4863709F453C0873709F08C
:1034600068C08E2D0E94921C52C09CE7980F903726
:1034700008F05FC08F770E94AB124EC08F010E5FC5
:103480001F4FFE01849190E2980F983050F487709E
:10349000FD2D01C0FF0F8A95EAF78F2F0E94981C1F
:1034A00015C00E94141214C08F010E5F1F4FFE0141
:1034B000849190E2980F983068F48770FD2D01C0D8
:1034C000FF0F8A95EAF78F2F0E949E1C0E94BF1C57
:1034D000E80122C00E94AB12FBCFCF010296FE0191
:1034E000C491CC2361F0EFE9FFE03197F1F700C020
:1034F0000000C150F6CFCF010296FE01F490EC011E
:103500000BC00E94821CE82E07C00E94951C0E94DE
:10351000BF1C02C00E9414128F2D882341F0EFE9D6
:10352000FFE03197F1F700C000008150F6CFFE01B7
:103530007CCFDF91CF911F910F91FF90EF90DF90A3
:1035400008956093290470932A0480932B04909328
:103550002C040C940D1D089560932D0470932E047B
:1035600080932F04909330040C940C1D0F931F93A1
:1035700000912D0410912E0420912F0430913004DD
:10358000602B712B822B932B60932D0470932E0450
:1035900080932F04909330041F910F910C940C1D75
:1035A0000F931F9300912D0410912E0420912F044E
:1035B00030913004602371238223932360932D0480
:1035C00070932E0480932F04909330041F910F91D9
:1035D0000C940C1D0F931F9300912D0410912E0439
:1035E00020912F0430913004602771278227932780
:1035F00060932D0470932E0480932F0490933004D5
:103600001F910F910C940C1D60E070E0CB010C94A5
:10361000A11A0F931F9341E050E060E070E08A012F
:103620009B0104C0000F111F221F331F8A95D2F780
:10363000C901B8011F910F910C94A11A0F931F9308
:1036400041E050E060E070E004C0440F551F661F89
:10365000771F8A95D2F78091290490912A04A0912E
:103660002B04B0912C048A019B01082B192B2A2BC7
:103670003B2BC901B8011F910F910C94A11A0F9314
:103680001F9341E050E060E070E004C0440F551F1C
:10369000661F771F8A95D2F7409550956095709573
:1036A0008091290490912A04A0912B04B0912C04BC
:1036B0008A019B01082319232A233B23C901B8014E
:1036C0001F910F910C94A11A0F931F9341E050E0AA
:1036D00060E070E004C0440F551F661F771F8A9595
:1036E000D2F78091290490912A04A0912B04B091E3
:1036F0002C048A019B01082719272A273B27C90187
:10370000B8011F910F910C94A11A0F931F93009170
:10371000290410912A0420912B0430912C04602B51
:10372000712B822B932B1F910F910C94A11A0F9345
:103730001F930091290410912A0420912B043091A9
:103740002C0460237123822393231F910F910C94E7
:10375000A11A0F931F930091290410912A0420911C
:103760002B0430912C0460277127822793271F9107
:103770000F910C94A11A08958F929F92AF92BF92CD
:10378000DF92EF92FF920F931F93CF93DF9300D0BE
:1037900000D01F92CDB7DEB76B837C838D838A0107
:1037A0008C819D81892B31F01F3F31F481E04F3FA7
:1037B00019F403C081E001C080E080FF03C080E015
:1037C00090E054C08B81882309F43DC08090290487
:1037D00090902A04A0902B04B0902C0480912D048A
:1037E00090912E04A0912F04B0913004882A992A38
:1037F000AA2ABB2A2FE1E22EF12CD501C4010E2CFE
:1038000004C0B695A795979587950A94D2F780FD41
:1038100006C081E0E81AF10880F7D12C07C0DE2C41
:10382000B8018E2D0E94FF1D019799F3E12FF0E062
:1038300093E0EE0FFF1F9A95E1F7E755FC4FE00F7D
:10384000F11DD0820CC0E12FF0E083E0EE0FFF1FEE
:103850008A95E1F7E755FC4FE00FF11DD080098311
:103860001A8369817A818D2D0E94FF1D0F900F9020
:103870000F900F900F90DF91CF911F910F91FF90BC
:10388000EF90DF90BF90AF909F908F900895209120
:10389000110130911201F90132969FEF40E05191F0
:1038A000851789F09F3F19F4511101C0942F4F5F84
:1038B0004630A9F79F3F39F0F901E90FF11D97FD57
:1038C000FA95828308950895E0911101F091120113
:1038D0009F012A5F3F4F9281891301C01282319666
:1038E000E217F307C1F7089581E090E0E09111013C
:1038F000F0911201E80FF91F1082019688309105AE
:10390000A9F7089580913B04089590913B04892B79
:1039100080933B040895809590913B048923809384
:103920003B04089580933B04089510923B0408954E
:1039300090913A04892B80933A0408958095909150
:103940003A04892380933A04089510923A04089522
:1039500080933104089510923104089580911101EB
:1039600090911201FC0131969C01285F3F4F80E04D
:10397000919191118F5FE217F307D1F70895E091CC
:103980001101F091120180913B048083E0911101BB
:10399000F0911201908180913A04892B808380916B
:1039A0003104882361F0E0911101F09112019081BE
:1039B000892B80830E94AE1C81111092310480916A
:1039C0001101909112010C942A1090933901809367
:1039D000380108958295982F9373292F220F220F73
:1039E000982F9C7C96959695922B892F8575880F9C
:1039F0009A7A9695892B08950895CF93DF9300D0F6
:103A000000D01F92CDB7DEB70F900F900F900F90A0
:103A10000F90DF91CF910895089508950C9481112E
:103A200080E0089580915104843021F110923D048A
:103A300020E488E190E00FB6F894A89580936000A8
:103A40000FBE2093600083B7817F846083BF83B7FC
:103A5000816083BF7894889583B78E7F83BF0FB6CC
:103A6000F894A8958091600088618093600010921E
:103A700060000FBE0895CF930E94CC110E94F10602
:103A80000E94CD11C0E08C2F0E94A007811104C0BC
:103A9000CF5FC031C1F701C081E0CF9108951F927F
:103AA0000F920FB60F9211248F939F93AF93BF93F2
:103AB00080913D04811113C080913E0490913F0498
:103AC000A0914004B09141044196A11DB11D809385
:103AD0003E0490933F04A0934004B0934104BF91EF
:103AE000AF919F918F910F900FBE0F901F901895DF
:103AF00082E084BD93E095BD9AEF97BD80936E0000
:103B000008952FB7F89480913E0490913F04A091BE
:103B10004004B09141042FBF08952FB7F8946091ED
:103B20003E0470913F0480914004909141042FBF66
:103B300008959C014FB7F89480913E0490913F0402
:103B4000A0914004B09141044FBF821B930B089594
:103B500078941F920F920FB60F9211248F939F9318
:103B6000AF93BF9380913E0490913F04A091400495
:103B7000B09141040196A11DB11D80933E04909324
:103B80003F04A0934004B0934104BF91AF919F9133
:103B90008F910F900FBE0F901F9018950E94F10EFD
:103BA000F89487E797E7909301088093000887E0EF
:103BB00090EBDC0180935A0490935B04A0935C0427
:103BC000B0935D049CE088E10FB6F894A8958093CB
:103BD00060000FBE90936000FFCFE92FF0E093E00C
:103BE000EE0FFF1F9A95E1F7E80FF11DE855FE4F24
:103BF0008491982F92959F708F7097700895CF93AE
:103C0000C82FCB010E94ED1D292F30E054E0220F78
:103C1000331F5A95E1F7282B203831051CF080E03E
:103C200090E018C0EC2FF0E023E0EE0FFF1F2A9584
:103C3000E1F79770E90FF11D34E0EE0FFF1F3A95A1
:103C4000E1F78F70E80FF11DEE0FFF1FE855FF4FF2
:103C500085919491CF91089580E090E00895089522
:103C60008091440480FF0CC08091160190E065E0D3
:103C700070E00E94FE2595958795959587952EC0B5
:103C800081FF0AC08091160190E065E070E00E941B
:103C9000FE259595879522C082FF08C08091160168
:103CA00090E065E070E00E94FE2518C02091450478
:103CB0002223D9F030911501231780F78091160146
:103CC00090E065E070E00E94FE25622F70E00E94A7
:103CD000FE25632F70E00E940F26CB0180389105EE
:103CE00038F4009739F481E005C085E090E008954C
:103CF0008FE7089508958091440480FF08C0609183
:103D0000140170E0759567957595679523C081FFDF
:103D100006C06091140170E0759567951BC082FF25
:103D200004C06091140170E012C0609145046623E4
:103D3000A9F0209113016217A0F78091140170E09F
:103D400090E00E94FE25622F70E00E940F266038EE
:103D5000710540F46115710519F406C061E070E069
:103D6000862F08958FE7089581E00895803F21F41C
:103D70000E94301E819504C0813F29F40E94301EAC
:103D8000809348040895823F21F40E94301E81955B
:103D900004C0833F29F40E94301E80934704089595
:103DA000893F19F40E947B1E05C08A3F31F40E94AE
:103DB0007B1E81958093490408958B3F21F40E94D6
:103DC0007B1E819504C08C3F29F40E947B1E80934A
:103DD0004A040895843F21F480914604816017C00D
:103DE000853F21F480914604826011C0863F21F412
:103DF0008091460484600BC0873F21F48091460483
:103E0000886005C0883F31F48091460480618093CA
:103E1000460408958D3F21F48091440481600BC0D5
:103E20008E3F21F480914404826005C08F3F29F4C5
:103E3000809144048460809344040895803F39F461
:103E40008091480487FF6CC01092480469C0813F8C
:103E500029F4809148041816BCF362C0909147047D
:103E6000823F29F497FF5CC01092470459C0833FFA
:103E700019F41916CCF354C0893F41F480914904D8
:103E800018160CF04DC0109249044AC08A3F29F41C
:103E90008091490487FF44C0F6CF8B3F39F480916D
:103EA0004A0487FF3DC010924A043AC08C3F29F46F
:103EB00080914A041816BCF333C0843F21F48091EA
:103EC00046048E7F17C0853F21F4809146048D7F84
:103ED00011C0863F21F4809146048B7F0BC0873F41
:103EE00021F480914604877F05C0883F31F480919A
:103EF00046048F7E8093460413C08D3F21F4809149
:103F000044048E7F0BC08E3F21F4809144048D7F4A
:103F100005C08F3F29F4809144048B7F8093440433
:103F20008091470481110EC08091480481110AC01C
:103F300080914904811106C080914A04811102C018
:103F400010924504089580913C0483FF7EC082EF67
:103F500094E00E94C105809146041F928F938DEEDC
:103F600094E09F938F930E945A068BEE94E00E94F8
:103F7000C10580914704282F082E000C330B3F9376
:103F80008F9388EE94E09F938F930E945A0686EE5B
:103F900094E00E94C10580914804282F082E000C4F
:103FA000330B3F938F9383EE94E09F938F930E9404
:103FB0005A0681EE94E00E94C10580914904282FA1
:103FC000082E000C330B3F938F938EED94E09F935C
:103FD0008F930E945A068CED94E00E94C105809157
:103FE0004A04282F082E000C330B3F938F9389ED42
:103FF00094E09F938F930E945A0686ED94E00E946E
:10400000C105809145041F928F9383ED94E09F93A7
:104010008F930E945A0681ED94E00E94C105809121
:1040200044041F928F938EEC94E09F938F930E9491
:104030005A068BEC94E00E94C1058DB79EB74C9652
:104040000FB6F8949EBF0FBE8DBF86E494E00E9429
:1040500073100E94811D909343048093420408953D
:104060001F93CF93DF9380914204909143040E9469
:10407000991DFC0120914504222321F08091170114
:1040800090E007C08091180190E06AE070E00E9423
:10409000FE25E817F90708F485C080914704C09110
:1040A0004804D091490410914A04811107C0C111FC
:1040B00075C0D11173C0111171C074C02F3F19F0B8
:1040C0002F5F20934504181624F40E94301E80931D
:1040D00047048091470487FF05C00E94301E8195E8
:1040E000809347041C1624F40E94301E80934804D9
:1040F0008091480487FF05C00E94301E81958093FF
:10410000480460914704662331F1C0914804CC23F0
:1041100011F1062E000C770B880B990B0E94FD24E1
:1041200023E333E343E35FE30E9461250E94C52458
:10413000609347046C2FCC0F770B880B990B0E9470
:10414000FD2423E333E343E35FE30E9461250E9400
:10415000C524609348041D1624F40E947B1E80939E
:1041600049048091490487FF05C00E947B1E819508
:1041700080934904111624F40E947B1E80934A0404
:1041800080914A0487FF05C00E947B1E8195809321
:104190004A04DF91CF911F910C94A31F2F3F09F088
:1041A0008FCFA0CFDF91CF911F910895E6E4F4E087
:1041B00085E0DF011D928A95E9F71092450410927F
:1041C0004404089585E197E00E94C1051F9281E0B3
:1041D0008F931F9285E08F9387EC96E09F938F9348
:1041E0000E945A060F900F900F900F900F900F9013
:1041F00008958330E9F128F4813061F0823009F1CB
:104200000895853009F462C008F449C0863009F485
:1042100074C0089580911801262F30E0280F311DB9
:104220002F3F310524F4680F6093180103C08FEF0E
:1042300080931801809118011F928F9380E096E07F
:1042400072C080911701262F30E0280F311D2F3FBB
:10425000310524F4680F6093170103C08FEF80933A
:104260001701809117011F928F938EEE95E05BC02E
:1042700080911601262F30E0280F311D2F3F310588
:1042800024F4680F6093160103C08FEF809316012A
:10429000809116011F928F938BED95E044C0809121
:1042A0001501262F30E0280F311D2F3F310524F452
:1042B000680F6093150103C08FEF80931501809103
:1042C00015011F928F9386EC95E02DC0809114010B
:1042D000262F30E0280F311D2F3F310524F4680FC1
:1042E0006093140103C08FEF809314018091140137
:1042F0001F928F938DEA95E016C080911301262FAF
:1043000030E0280F311D2F3F310524F4680F6093F2
:10431000130103C08FEF80931301809113011F924B
:104320008F9382E995E09F938F930E945A060F9096
:104330000F900F900F900895833081F128F4813011
:1043400059F08230D1F00895853009F449C0B8F1B0
:10435000863009F456C0089580911801681720F43A
:10436000861B8093180102C01092180180911801D9
:104370001F928F9383E895E054C0809117016817CE
:1043800020F4861B8093170102C0109217018091C0
:1043900017011F928F9381E795E043C0809116012A
:1043A000681720F4861B8093160102C01092160134
:1043B000809116011F928F938EE595E032C0809117
:1043C0001501681720F4861B8093150102C0109216
:1043D0001501809115011F928F9389E495E021C00A
:1043E00080911401681720F4861B8093140102C089
:1043F00010921401809114011F928F9380E395E035
:1044000010C080911301681720F4861B809313015C
:1044100002C010921301809113011F928F9385E1C6
:1044200095E09F938F930E945A060F900F900F90E4
:104430000F900895CF93C82F1F928F938AE198E031
:104440009F938F930E945A0681E090E0A0E0B0E035
:10445000BC01CD0104C0660F771F881F991FCA9544
:10446000D2F70E94AC1A0F900F900F900F90CF913F
:104470000C942713CF93873288F58E3108F00BC147
:104480008E3009F487C0D8F4873009F460C08B30CF
:1044900009F44FC0863009F002C180913C04817F4D
:1044A0008E7F80933C048FE198E00E94C10581EDEE
:1044B0009AE00E94C10581E080934C0446C0863199
:1044C00009F4B0C020F4803109F47AC0E8C0893121
:1044D00009F491C08B3109F449C0E1C0883349F136
:1044E00050F4893209F4D5C0853309F4D2C087323B
:1044F00009F0D5C0CEC0833409F4CBC028F48A3388
:1045000008F4CDC08953C8C0883409F0C8C00E94DF
:10451000271380EC9AE00E94C1052FEF83ED90E312
:10452000215080409040E1F700C000000E94CE1D65
:104530000CC086E498E041C087EA9AE00E94C10579
:1045400080913C04816080933C04C1E0ADC08091C7
:104550003C04C82FC17080FFEFCF83EB9AE00E942C
:10456000C10580913C04817F8E7F3FC090913C04C7
:1045700091FBCC27C0F981E0C827892FC0FB81F9C6
:1045800080933C04CC2319F08AE99AE029C08CE896
:104590009AE013C090913C0492FBCC27C0F981E0D3
:1045A000C827892FC0FB82F980933C04CC2319F0E3
:1045B0008DE79AE015C08DE69AE00E94C105C5CF4F
:1045C00090913C0493FBCC27C0F981E0C827892F48
:1045D000C0FB83F980933C04CC2351F081E69AE040
:1045E0000E94C10580913C04816080933C045CC0C2
:1045F00084E59AE0E2CF85E49AE00E94C10585E176
:104600009AE00E94C1058FEC99E00E94C10586EAFC
:1046100099E00E94C10580E799E00E94C10584E409
:1046200099E0CBCF86E399E00E94C1050E941E105D
:104630001F928F938CE199E09F938F930E945A066B
:10464000809110011F928F9385E099E09F938F9343
:104650000E945A06809159031F928F9382EF98E02F
:104660009F938F930E945A060E948D1D9F938F9354
:104670007F936F938BED98E09F938F930E945A06E0
:104680008DB79EB742960FB6F8949EBF0FBE8DBFF2
:104690005CCF80E001C08D510E941A2256CF89ED77
:1046A00098E00E94C105C0E08C2FCF91089580E072
:1046B00008950C9457230F931F93CF93C82F809185
:1046C0004C048130B1F020F0823009F45BC052C15B
:1046D00060E070E08CE090E00E948411892BC9F4C6
:1046E000E0911101F09112018081843409F044C1FC
:1046F00010C060E070E08CE090E00E9484118C01BA
:10470000892B39F4E0911101F091120180818434F8
:1047100061F48C2F0E945923811104C08C2F0E94B8
:104720003A222EC081E090E02BC08C2F0E945723AC
:10473000811124C1C431E1F070F4CB3081F0C0317B
:10474000D1F40E94E22082E198E00E94C10582E05B
:1047500080934C0413C1C93259F0C83361F48FE11E
:1047600098E00E94C10586E198E00E94C10506C15B
:1047700010924C0404C080E198E00E94C105802F93
:104780008170FFC0C43228F5CE3108F0C1C0CB30F3
:10479000A1F1D0F4C73009F0D3C08EE180931801A5
:1047A00082E3809317018AE08093160184E180936D
:1047B000150188E08093140188E28093130186EB51
:1047C00096E00E94C105BFC0C33149F1C431C1F0B8
:1047D000B7C0CB3409F4A9C028F4C93289F0C83372
:1047E00061F0AEC0C13509F49EC0C23509F499C06C
:1047F000CE3409F0A5C06AE09EC00E94E220A3C0AA
:1048000080914B04882319F010924B049CC083ECD8
:1048100096E00E94C10581E080934C04B2C08DE90E
:1048200096E00E94C1058BE896E00E94C105809148
:1048300018011F928F9388E896E09F938F930E94B0
:104840005A0686E896E00E94C10584E796E00E9439
:10485000C105809117011F928F9381E796E09F9386
:104860008F930E945A068FE696E00E94C10580E66B
:1048700096E00E94C105809116011F928F938DE5ED
:1048800096E09F938F930E945A068BE596E00E94D4
:10489000C1058AE496E00E94C105809115011F922E
:1048A0008F9387E496E09F938F930E945A0685E446
:1048B00096E00E94C10580E396E00E94C1058091C8
:1048C00014011F928F938DE296E09F938F930E9425
:1048D0005A068BE296E00E94C10584E196E00E94B0
:1048E000C105809113011F928F9381E196E09F9300
:1048F0008F930E945A068FE096E00E94C1058DB703
:104900009EB748960FB6F8949EBF0FBE8DBF1BC0D2
:10491000CE51EC2FF0E0E25DFE4F808180934B049E
:1049200012C061E003C061E006C06AE080914B0400
:104930000E94F92008C080914B040E949C2103C072
:1049400084EB96E013C080914B04882369F01F929A
:104950008F938EEA96E09F938F930E945A060F9052
:104960000F900F900F9004C08BEA96E00E94C10553
:1049700081E007C010924C0480E003C001E010E029
:10498000FECECF911F910F9108950E94CC24689480
:10499000B1110C945B2508950E94402588F09F5723
:1049A00098F0B92F9927B751B0F0E1F0660F771F53
:1049B000881F991F1AF0BA95C9F714C0B13091F049
:1049C0000E945A25B1E008950C945A25672F782F3C
:1049D0008827B85F39F0B93FCCF38695779567950E
:1049E000B395D9F73EF490958095709561957F4F7A
:1049F0008F4F9F4F0895E89409C097FB3EF4909520
:104A00008095709561957F4F8F4F9F4F9923A9F0A7
:104A1000F92F96E9BB279395F69587957795679536
:104A2000B795F111F8CFFAF4BB0F11F460FF1BC07A
:104A30006F5F7F4F8F4F9F4F16C0882311F096E90D
:104A400011C0772321F09EE8872F762F05C06623BB
:104A500071F096E8862F70E060E02AF09A95660F74
:104A6000771F881FDAF7880F9695879597F908952D
:104A700057FD9058440F551F59F05F3F71F047950F
:104A8000880F97FB991F61F09F3F79F087950895F4
:104A9000121613061406551FF2CF4695F1DF08C013
:104AA000161617061806991FF1CF86957105610530
:104AB00008940895E894BB2766277727CB0197F9D8
:104AC00008950E9473250C94ED250E94DF2538F08F
:104AD0000E94E62520F0952311F00C94D6250C9425
:104AE000DC250C945B250E94382578F39923C9F3C3
:104AF0005523B9F3950F50E0551FAA27EE27FF273E
:104B0000BB2700240894679520F4E20FF31FB41F1D
:104B10000A1E220F331F441FAA1F6695A9F7779517
:104B200030F4F30FB41F0A1E121E08F46395330FFE
:104B3000441FAA1F221F769599F7879520F4B40F7A
:104B40000A1E121E631F440FAA1F221F331F8695C1
:104B5000A9F7862F712D602D11249F5750409AF090
:104B6000F1F088234AF0EE0FFF1FBB1F661F771F6F
:104B7000881F91505040A9F79E3F510580F00C943A
:104B8000D6250C945B255F3FE4F3983ED4F38695DD
:104B900077956795B795F795E7959F5FC1F7FE2BDA
:104BA000880F911D9695879597F9089597F99F67B6
:104BB00080E870E060E008959FEF80EC08950024A5
:104BC0000A941616170618060906089500240A9472
:104BD00012161306140605060895092E0394000CF8
:104BE00011F4882352F0BB0F40F4BF2B11F460FF87
:104BF00004C06F5F7F4F8F4F9F4F0895002455274C
:104C000004C0080E591F880F991F009729F0769548
:104C10006795B8F37105B9F7802D952F089597FB27
:104C2000072E16F4009407D077FD09D00E9429269C
:104C300007FC05D03EF4909581959F4F089570959F
:104C400061957F4F0895EE0FFF1F0590F491E02DC1
:104C50000994AA1BBB1B51E107C0AA1FBB1FA617C3
:104C6000B70710F0A61BB70B881F991F5A95A9F715
:0E4C700080959095BC01CD010895F894FFCF7A
:104C7E000550020000FF3208C2089F086908350877
:104C8E000132042808140A321E404D36223704EA37
:104C9E0003B40392031E033703500369030001029A
:084CAE000304050607080900D4
:00000001FF
